:100000000C9462000C948A000C948A000C948A0070
:100010000C948A000C948A000C948A000C948A0038
:100020000C948A000C948A000C948A000C948A0028
:100030000C948A000C948A000C948A000C948A0018
:100040000C94E2050C948A000C943C080C948A00F1
:100050000C948A000C948A000C948A000C948A00F8
:100060000C948A000C948A000000000024002700F1
:100070002A0000000000250028002B0000000000DE
:1000800023002600290004040404040404040202DA
:100090000202020203030303030301020408102007
:1000A0004080010204081020010204081020000012
:1000B0000007000201000003040600000000000029
:1000C00000000D0A11241FBECFEFD4E0DEBFCDBF6C
:1000D00011E0A0E0B1E0ECE3F5E102C005900D9283
:1000E000A634B107D9F712E0A6E4B1E001C01D9231
:1000F000A232B107E1F710E0C4ECD0E004C02297CF
:10010000FE010E94990AC23CD107C9F70E94FE0471
:100110000C949D0A0C940000FB01DC0104C08D913D
:100120000190801921F441505040C8F7881B990B69
:1001300008958091550180936201809156018093CA
:1001400063018091570180936401109265010895C5
:1001500020E030E0F901E85AFE4FD901A25BBE4F22
:100160008C9180832F5F3F4F2A30310599F7809122
:100170005F018093620180916001809363018091AF
:10018000610180936401109265010895EF92FF92DE
:100190000F931F93CF93DF93809146019091470176
:1001A000181619061CF0C0E0D0E045C0EE24FF246C
:1001B00087012CC061E0809108010E947705809141
:1001C00046019091470162E070E00E94330ACB0142
:1001D0000E94360660E0809108010E9477058091B8
:1001E00046019091470162E070E00E94330ACB0122
:1001F0000E9436068091460190914701AA2797FDFB
:10020000A095BA2FE80EF91E0A1F1B1F80914A0104
:1002100090914B01A0914C01B0914D01E816F90667
:100220000A071B073CF20EC080914A0190914B01D6
:100230000E943606219680912C0190912D01C817BD
:10024000D90794F3DF91CF911F910F91FF90EF9019
:100250000895EF92FF920F931F93CF93DF938EE158
:10026000E82E81E0F82E00E211E0C0E0D0E02FC0DF
:10027000F701819191917F0190934701809346010D
:10028000F801619171918F01709349016093480168
:10029000882777FD8095982F20912601309127019E
:1002A00040912801509129010E94140A60934A014B
:1002B00070934B0180934C0190934D010E94C600B6
:1002C00080912A0190912B010E94360621968091FF
:1002D000240190912501C817D90754F2DF91CF91DD
:1002E0001F910F91FF90EF900895EF92FF920F935F
:1002F0001F93CF93DF932AE0E22E21E0F22E04E158
:1003000011E0C0E0D0E02FC0F701819191917F0111
:100310009093470180934601F801619171918F019B
:100320007093490160934801882777FD8095982F45
:1003300020912601309127014091280150912901F7
:100340000E94140A60934A0170934B0180934C0100
:1003500090934D010E94C60080912A0190912B013B
:100360000E94360621968091220190912301C817A0
:10037000D90754F2DF91CF911F910F91FF90EF9029
:100380000895FF920F931F93CF93DF938B01F82E65
:1003900061E00E940905C0E0D0E015C061E08F2D4A
:1003A0000E94770568EC70E080E090E00E947D0696
:1003B00060E08F2D0E94770568EC70E080E090E0AF
:1003C0000E947D062196C017D10744F3DF91CF919B
:1003D0001F910F91FF900895AF92BF92CF92DF923D
:1003E000EF92FF920F931F930E942A06609372016F
:1003F000709373018093740190937501209176013D
:10040000309177014091780150917901621B730B13
:10041000840B950B9B01AC0197FF07C0509540954D
:10042000309521953F4F4F4F5F4F20937A01309386
:100430007B0140937C0150937D0180912E0190912E
:100440002F01A0913001B091310182179307A407C9
:10045000B5070CF07FC0809134010E94C4059093D1
:100460006701809366018756924014F460E001C0F2
:1004700061E0809132010E94770540910601509120
:100480000701662757FD6095762F2AE030E08FE060
:1004900092E00E94FA076091380170913901882733
:1004A00077FD8095982F0E947D0660E071E08FE0D7
:1004B00092E00E94340760913801709139018827D9
:1004C00077FD8095982F0E947D066091660170915E
:1004D0006701882777FD8095982F2AE233E040E076
:1004E00050E05F934F933F932F93AA24BB24650161
:1004F0005CE5E52E53E0F52E012D112D20E030E0D6
:1005000040E050E00E94A706AB01BC012AE030E0C9
:100510008FE092E00E94FA076091380170913901F2
:10052000882777FD8095982F0E947D068091720123
:1005300090917301A0917401B0917501809376013F
:1005400090937701A0937801B09379010F900F9069
:100550000F900F901F910F91FF90EF90DF90CF9031
:10056000BF90AF900895EF92FF920F931F93CF9398
:10057000DF931092710110927001CFE0D2E068E534
:10058000E62E61E0F62E0EE411E029C0CE010E94B5
:100590009C099093670180936601209170013091CE
:1005A0007101F901E25BFE4F80832F5F3F4F309373
:1005B0007101209370012A30310589F44AE050E03E
:1005C000B701C8010E948C00892B19F40E942901EF
:1005D00006C00E94A8000E9499000E947501CE01E9
:1005E0000E948509882391F6DF91CF911F910F9189
:1005F000FF90EF9008952F923F924F925F926F92EB
:100600007F928F929F92AF92BF92CF92DF92EF92A2
:10061000FF920F931F9340918001509181016627B3
:1006200057FD6095762FBFE08B2EB2E09B2E2AE01F
:1006300030E0C4010E94FA076091380170913901DD
:10064000882777FD8095982F0E947D06A4E02A2EAA
:10065000A1E03A2EB101C4010E9434076091380133
:1006600070913901882777FD8095982F0E947D062B
:1006700062E671E0C4010E94340760913801709114
:100680003901882777FD8095982F0E947D06B1015A
:10069000C4010E94340760913801709139018827A4
:1006A00077FD8095982F0E947D066091680170917A
:1006B0006901882777FD8095982FFFEF4F2E512CE9
:1006C000612C712C7F926F925F924F92AA24BB246F
:1006D0006501E3EAEE2EE2E0FE2E012D112D20E071
:1006E00030E040E050E00E94A706AB01BC012AE0E8
:1006F00030E0C4010E94FA0760913801709139011D
:10070000882777FD8095982F0E947D06B101C4014E
:100710000E9434076091380170913901882777FD74
:100720008095982F0E947D0660916A0170916B01FF
:10073000882777FD8095982F7F926F925F924F92D6
:1007400020E030E040E050E00E94A706AB01BC0191
:100750002AE030E0C4010E94FA07609138017091EC
:100760003901882777FD8095982F0E947D06B10179
:10077000C4010E94340760913801709139018827C3
:1007800077FD8095982F0E947D0660916C01709195
:100790006D01882777FD8095982F7F926F925F92E9
:1007A0004F9220E030E040E050E00E94A706AB010D
:1007B000BC012AE030E0C4010E94FA0760913801D0
:1007C00070913901882777FD8095982F0E947D06CA
:1007D000B101C4010E943407609138017091390160
:1007E000882777FD8095982F0E947D0660916E0185
:1007F00070916F01882777FD8095982F7F926F9277
:100800005F924F9220E030E040E050E00E94A70667
:10081000AB01BC012AE030E0C4010E940A086091EB
:10082000380170913901882777FD8095982F0E94B3
:100830007D068DB79EB740960FB6F8949EBF0FBE4B
:100840008DBF1F910F91FF90EF90DF90CF90BF90E1
:10085000AF909F908F907F906F905F904F903F9060
:100860002F90089580E00E94C405909369018093C1
:10087000680181E00E94C40590936B0180936A0136
:1008800082E00E94C40590936D0180936C0184E026
:100890000E94C40590936F0180936E010E94FB0239
:1008A00008950E94B3020E9432040E94EC0164E6A3
:1008B00070E080E090E00E947D06089561E0809104
:1008C00036010E94770561E0809108010E940905C8
:1008D00040E855E260E070E08FE092E00E9494080A
:1008E00061E0809132010E94090561E0809136014A
:1008F0000E94090585E090E008C060E00E940905BB
:1009000080917E0190917F01019690937F01809369
:100910007E0180917E0190917F01893091056CF379
:1009200085E090E034C00E942905892B59F180911F
:100930007E0190917F018530910519F481E090E06E
:100940000FC08630910519F482E090E009C087302D
:10095000910519F484E090E003C08830910521F4FA
:10096000909367018093660180918001909181014D
:100970002091660130916701820F931F909381014E
:100980008093800180917E0190917F0101969093E8
:100990007F0180937E0180917E0190917F0189305B
:1009A00091050CF285E190E09093810180938001A4
:1009B00063E070E08DE090E00E94C1010E9475014B
:1009C00080E38093620180936301809364011092BD
:1009D000650120E030E0F901E25BFE4F80E38083B7
:1009E000F901E85AFE4F80832F5F3F4F29303105D0
:1009F00091F710925701109261010895CFEFD4E062
:100A0000DEBFCDBF0E9443060E945E040E945104D7
:100A1000FDCF282F3327C90186569F4FFC019491A3
:100A20002A573F4FF9018491882391F0E82FFF273F
:100A3000EE0FFF1FE859FF4FA591B491662329F4EB
:100A40008C91909589238C9308958C91892B8C930C
:100A50000895482F5527CA0182559F4FFC012491C4
:100A6000CA0186569F4FFC0194914A575F4FFA0185
:100A70003491332319F480E090E00895222331F17A
:100A8000233021F4809180008F7705C0243031F429
:100A9000809180008F7D8093800018C0213019F4F0
:100AA00084B58F7704C0223021F484B58F7D84BD56
:100AB0000DC0263021F48091B0008F7705C027301B
:100AC00029F48091B0008F7D8093B000E32FFF2741
:100AD000EE0FFF1FE458FF4FA591B4918C9120E0D9
:100AE00030E0892311F021E030E0C9010895482F5A
:100AF0005527CA0182559F4FFC012491CA01865691
:100B00009F4FFC0194914A575F4FFA013491332370
:100B1000D1F1222331F1233021F4809180008F77AD
:100B200005C0243031F4809180008F7D8093800057
:100B300018C0213019F484B58F7704C0223021F415
:100B400084B58F7D84BD0DC0263021F48091B00026
:100B50008F7705C0273029F48091B0008F7D809376
:100B6000B000E32FFF27EE0FFF1FEE58FF4FA591B8
:100B7000B491662329F48C91909589238C930895E0
:100B80008C91892B8C9308958F7090913A01929556
:100B9000990F990F907C982B90937C0080917A000C
:100BA000806480937A0080917A0086FDFCCF20914A
:100BB0007800809179009927982F88273327822BF6
:100BC000932B08951F920F920FB60F9211242F931B
:100BD0003F938F939F93AF93BF93809186019091A2
:100BE0008701A0918801B091890130918A01019615
:100BF000A11DB11D232F2D5F2D3720F02D570196FC
:100C0000A11DB11D20938A018093860190938701D5
:100C1000A0938801B0938901809182019091830112
:100C2000A0918401B09185010196A11DB11D809311
:100C3000820190938301A0938401B0938501BF91B9
:100C4000AF919F918F913F912F910F900FBE0F9079
:100C50001F9018952FB7F8946091860170918701C5
:100C600080918801909189012FBF0895019751F0DB
:100C7000880F991F880F991F02972FB7F894019733
:100C8000F1F72FBF0895789484B5826084BD84B550
:100C9000816084BD85B5826085BD85B5816085BD77
:100CA000EEE6F0E0808181608083E1E8F0E0808121
:100CB00082608083808181608083E0E8F0E08081D1
:100CC00081608083E1EBF0E0808184608083E0EBF1
:100CD000F0E0808181608083EAE7F0E080818460D9
:100CE0008083808182608083808181608083808135
:100CF000806880831092C1000895EF92FF920F9355
:100D00001F937B018C018FB7F8944091860150911D
:100D1000870160918801709189018FBF2FB7F89486
:100D20008091860190918701A0918801B0918901FD
:100D30002FBF841B950BA60BB70BE816F9060A0705
:100D40001B0760F71F910F91FF90EF9008952F926E
:100D50003F924F925F926F927F928F929F92AF924B
:100D6000BF92CF92DF92EF92FF920F931F93CF9398
:100D7000DF93CDB7DEB73B014C0119012A016D8924
:100D80007E898F89988D6A197B098C099D09621A61
:100D9000730A840A950AA40193010E94140AE218B6
:100DA000F30804091509A80197010E94680A2A0D91
:100DB0003B1D4C1D5D1DCA01B901DF91CF911F91F3
:100DC0000F91FF90EF90DF90CF90BF90AF909F90EA
:100DD0008F907F906F905F904F903F902F900895ED
:100DE0000F931F93CF93DF938C01EB0109C02196E2
:100DF000D801ED91FC910190F081E02DC801099599
:100E000068816623A1F7DF91CF911F910F9108951B
:100E1000EF92FF920F931F93CF93DF938C017B018F
:100E2000EA010BC0D7016D917D01D801ED91FC91D4
:100E30000190F081E02DC80109952197BFEFCF3FC8
:100E4000DB0781F7DF91CF911F910F91FF90EF901A
:100E50000895DC01ED91FC910190F081E02D099560
:100E600008950E9429070895DC01ED91FC9102800C
:100E7000F381E02D099508950F931F938C016DE088
:100E80000E9431076AE0C8010E9431071F910F914B
:100E900008952F923F924F925F926F927F928F921E
:100EA0009F92AF92BF92CF92DF92EF92FF920F93F9
:100EB0001F93CF93DF93CDB7DEB7A2970FB6F89409
:100EC000DEBF0FBECDBF9AA389A36A017B01411586
:100ED00051056105710521F460E30E9431074EC0A0
:100EE000882499245401422E5524662477241E0117
:100EF0000894211C311C8101080D191DC701B60180
:100F0000A30192010E94460AF80160830894811CA3
:100F1000911CA11CB11CC701B601A30192010E9442
:100F2000460A69017A01211531054105510519F774
:100F3000089481089108A108B1087101E80CF91C16
:100F40000894811C911CA11CB11C13C00894810839
:100F50009108A108B108F70160816A3010F4605D62
:100F600001C0695C89A19AA10E9431070894E10837
:100F7000F10881149104A104B10441F7A2960FB6BF
:100F8000F894DEBF0FBECDBFDF91CF911F910F91BF
:100F9000FF90EF90DF90CF90BF90AF909F908F9099
:100FA0007F906F905F904F903F902F900895EF92B9
:100FB000FF920F931F93CF93DF93EC017A018B0184
:100FC00077FF0BC06DE20E94310710950095F094F9
:100FD000E094E11CF11C011D111D2AE0B801A701DC
:100FE000CE010E944907DF91CF911F910F91FF9091
:100FF000EF9008952115310521F4642F0E943107E7
:1010000008952A30310519F40E94D70708950E94E7
:10101000490708950F931F938C010E94FA07C80196
:101020000E943C071F910F9108950F931F93CF9338
:10103000DF93482FFB018B0100581F4FD801CD9142
:10104000DC91CE01019660E870E00E94330A9C01B9
:10105000EE57FF4F80819181E258F0402817390701
:1010600031F0CE0FDF1F4883F80131832083DF91F9
:10107000CF911F910F9108951F920F920FB60F926B
:1010800011242F933F934F935F936F937F938F938D
:101090009F93AF93BF93EF93FF938091C6006BE84C
:1010A00071E00E941508FF91EF91BF91AF919F9160
:1010B0008F917F916F915F914F913F912F910F9001
:1010C0000FBE0F901F9018958F92AF92CF92DF9224
:1010D000EF92FF920F931F93CF93DF93CDB7DEB7BD
:1010E000FC018FE391E09183808373836283558356
:1010F00044833783268311870087F386E286D5866B
:10110000C486A68687868D85808B8E85818B8F850C
:10111000828BDF91CF911F910F91FF90EF90DF9025
:10112000CF90AF908F9008956F927F928F929F9201
:10113000AF92BF92CF92DF92EF92FF920F931F93E5
:10114000CF93DF93EC017A018B01415452446F40FD
:1011500070400CF07AC060E874E88EE190E0A8017D
:1011600097010E94680A2150304040405040CA0117
:10117000B90122E030E040E050E00E94680A4901F5
:101180005A012F5F3F4F4F4F5F4F64E0220F331FD5
:10119000441F551F6A95D1F760E074E284EF90E038
:1011A0000E94680ACA01B9012FEF30E040E050E028
:1011B0000E94140AA80197010E94680A4FEF642E4A
:1011C000712C6301C21AD30AD7FE04C0D094C19413
:1011D000D108D39460E079E08DE390E0A801970115
:1011E0000E94680A2150304040405040CA01B90175
:1011F00022E030E040E050E00E94680A2F5F3F4F5D
:101200004F4F5F4F93E0220F331F441F551F9A9596
:10121000D1F760E074E284EF90E00E94680ACA01AE
:10122000B9012FEF30E040E050E00E94140AA8011D
:1012300097010E94680AC301821B930B97FF03C0AA
:10124000909581959F4F8C1500F5E885F98581E093
:1012500090E00A8802C0880F991F0A94E2F7808301
:1012600060E079E08DE390E0A80197010E94680AB0
:101270002150304040405040CA01B90122E030E0E6
:1012800040E050E00E94680A04C0E885F9851082B9
:101290009401EC81FD81832F99278083EE81FF816A
:1012A0002083EA85FB85208141E050E0CA010E845D
:1012B00002C0880F991F0A94E2F7282B2083EA8541
:1012C000FB852081CA010F8402C0880F991F0A94F0
:1012D000E2F7282B2083EA85FB858081088802C0FD
:1012E000440F551F0A94E2F7842B8083DF91CF913E
:1012F0001F910F91FF90EF90DF90CF90BF90AF9034
:101300009F908F907F906F900895CF93DF93EC0123
:10131000EA81FB81E058FF4F8191919180589F4F66
:1013200020813181821B930B60E870E00E94330AB8
:101330009927DF91CF910895CF93DF93EC01EA8154
:10134000FB81EF01CE57DF4F48815981E058FF4FB5
:1013500080819181E058F0408417950719F48FEF50
:101360009FEF0DC0E40FF51F2081CA01019660E8D0
:1013700070E00E94330A99838883822F9927DF9136
:10138000CF910895CF93DF93DC01ED01E885F985D6
:1013900080819927098802C0959587950A94E2F77C
:1013A00080FFF3CFEC85FD856083DF91CF910895B9
:1013B0008F92AF92CF92DF92EF92FF920F931F9393
:1013C000019711F56F5F7F4FF9F481E08F9385E00E
:1013D0008F9387E08F93A3E08A2EF4E0AF2EE6ECA4
:1013E000CE2ED12C71ECE72EF12C00EC10E024EC89
:1013F00030E045EC50E06BE871E08FE092E00E9455
:1014000064080F900F900F901F910F91FF90EF9035
:10141000DF90CF90AF908F9008956FEF7FEF81E0D6
:1014200090E00E94D8090895629FD001739FF00157
:10143000829FE00DF11D649FE00DF11D929FF00D64
:10144000839FF00D749FF00D659FF00D9927729F9B
:10145000B00DE11DF91F639FB00DE11DF91FBD0126
:10146000CF011124089597FB092E07260AD077FD96
:1014700004D049D006D000201AF4709561957F4FB2
:101480000895F6F7909581959F4F0895A1E21A2E41
:10149000AA1BBB1BFD010DC0AA1FBB1FEE1FFF1F18
:1014A000A217B307E407F50720F0A21BB30BE40B68
:1014B000F50B661F771F881F991F1A9469F76095AF
:1014C0007095809590959B01AC01BD01CF01089569
:1014D00097FB092E05260ED057FD04D0D7DF0AD082
:1014E000001C38F450954095309521953F4F4F4F53
:1014F0005F4F0895F6F790958095709561957F4FB1
:101500008F4F9F4F0895AA1BBB1B51E107C0AA1F15
:10151000BB1FA617B70710F0A61BB70B881F991F94
:101520005A95A9F780959095BC01CD010895EE0FCD
:0C153000FF1F0590F491E02D0994FFCFFF
:10153C003A633A003A00110009007807EC07F60903
:10154C007807000010001000100008002000F60EB4
:10155C0020000500010010270000E8036400881338
:10156C0000000D000300040003000100000000C295
:06157C0009F0060807005B
:00000001FF
